BL51 BANKED LINKER/LOCATER V6.22                                                        08/27/2014  12:29:25  PAGE 1


BL51 BANKED LINKER/LOCATER V6.22, INVOKED BY:
C:\KEIL\C51\BIN\BL51.EXE miaobiao.obj TO miaobiao1


MEMORY MODEL: SMALL


INPUT MODULES INCLUDED:
  miaobiao.obj (MIAOBIAO)
  C:\KEIL\C51\LIB\C51S.LIB (?C_STARTUP)
  C:\KEIL\C51\LIB\C51S.LIB (?C_INIT)


LINK MAP OF MODULE:  miaobiao1 (MIAOBIAO)


            TYPE    BASE      LENGTH    RELOCATION   SEGMENT NAME
            -----------------------------------------------------

            * * * * * * *   D A T A   M E M O R Y   * * * * * * *
            REG     0000H     0008H     ABSOLUTE     "REG BANK 0"
            DATA    0008H     000EH     UNIT         ?DT?MIAOBIAO
            IDATA   0016H     0001H     UNIT         ?STACK

            * * * * * * *   C O D E   M E M O R Y   * * * * * * *
            CODE    0000H     0003H     ABSOLUTE     
            CODE    0003H     0005H     UNIT         ?PR?DELAY?MIAOBIAO
                    0008H     0003H                  *** GAP ***
            CODE    000BH     0003H     ABSOLUTE     
            CODE    000EH     008CH     UNIT         ?C_C51STARTUP
            CODE    009AH     003CH     UNIT         ?PR?TIMER0?MIAOBIAO
            CODE    00D6H     0023H     UNIT         ?PR?DISPLAY?MIAOBIAO
            CODE    00F9H     0019H     UNIT         ?C_INITSEG
            CODE    0112H     0014H     UNIT         ?PR?MAIN?MIAOBIAO



OVERLAY MAP OF MODULE:   miaobiao1 (MIAOBIAO)


SEGMENT
  +--> CALLED SEGMENT
---------------------
?C_C51STARTUP
  +--> ?PR?MAIN?MIAOBIAO
  +--> ?C_INITSEG

?PR?MAIN?MIAOBIAO
  +--> ?PR?DISPLAY?MIAOBIAO

?PR?DISPLAY?MIAOBIAO
  +--> ?PR?DELAY?MIAOBIAO



SYMBOL TABLE OF MODULE:  miaobiao1 (MIAOBIAO)

  VALUE           TYPE          NAME
BL51 BANKED LINKER/LOCATER V6.22                                                      08/27/2014  12:29:25  PAGE 2


  ----------------------------------

  -------         MODULE        MIAOBIAO
  C:0000H         SYMBOL        _ICE_DUMMY_
  D:00A0H         PUBLIC        P2
  D:00B0H         PUBLIC        P3
  D:0008H         PUBLIC        counter
  B:00A8H.7       PUBLIC        EA
  D:0009H         PUBLIC        number
  C:0003H         PUBLIC        delay
  D:000AH         PUBLIC        number_0
  D:000BH         PUBLIC        number_1
  C:0112H         PUBLIC        main
  D:0089H         PUBLIC        TMOD
  D:000CH         PUBLIC        tab
  B:00A8H.1       PUBLIC        ET0
  D:008CH         PUBLIC        TH0
  D:008AH         PUBLIC        TL0
  C:009AH         PUBLIC        timer0
  B:0088H.4       PUBLIC        TR0
  C:00D6H         PUBLIC        display
  -------         PROC          MAIN
  C:0112H         LINE#         7
  C:0112H         LINE#         8
  C:0112H         LINE#         9
  C:0115H         LINE#         10
  C:0118H         LINE#         11
  C:011BH         LINE#         12
  C:011DH         LINE#         13
  C:011FH         LINE#         14
  C:0121H         LINE#         15
  C:0121H         LINE#         16
  C:0121H         LINE#         17
  C:0124H         LINE#         18
  -------         ENDPROC       MAIN
  -------         PROC          DISPLAY
  C:00D6H         LINE#         21
  C:00D6H         LINE#         22
  C:00D6H         LINE#         23
  C:00DEH         LINE#         24
  C:00E1H         LINE#         25
  C:00E4H         LINE#         26
  C:00E7H         LINE#         27
  C:00EFH         LINE#         28
  C:00F2H         LINE#         29
  C:00F5H         LINE#         30
  C:00F8H         LINE#         31
  -------         ENDPROC       DISPLAY
  -------         PROC          TIMER0
  C:009AH         LINE#         33
  C:00A0H         LINE#         35
  C:00A2H         LINE#         36
  C:00A5H         LINE#         37
  C:00A8H         LINE#         38
  C:00AAH         LINE#         39
  C:00AFH         LINE#         40
  C:00AFH         LINE#         41
BL51 BANKED LINKER/LOCATER V6.22                                                      08/27/2014  12:29:25  PAGE 3


  C:00B2H         LINE#         42
  C:00B4H         LINE#         43
  C:00B9H         LINE#         44
  C:00B9H         LINE#         45
  C:00BCH         LINE#         46
  C:00BCH         LINE#         47
  C:00C4H         LINE#         48
  C:00CDH         LINE#         49
  C:00CDH         LINE#         50
  C:00CFH         LINE#         51
  -------         ENDPROC       TIMER0
  -------         PROC          DELAY
  -------         DO            
  D:0007H         SYMBOL        i
  -------         ENDDO         
  C:0003H         LINE#         52
  C:0003H         LINE#         53
  C:0003H         LINE#         55
  C:0007H         LINE#         56
  -------         ENDPROC       DELAY
  -------         ENDMOD        MIAOBIAO

Program Size: data=23.0 xdata=0 code=291
LINK/LOCATE RUN COMPLETE.  0 WARNING(S),  0 ERROR(S)
